:100000001B29A801AA01A90001300828A900043071
:10001000A5002A082802031D0F28290827020430FA
:1000200003180130031902302505031D013017297B
:100030008030A100FE30BB200130BB207530A8000D
:100040003030E728A101A117B000FE30BB203008F6
:10005000BB28A401AB00AC01A01124080319A01512
:100060001030A3000301AB0DAC0D031801305C2070
:100070002308031D32280800A401AB00AC01A01125
:1000800024080319A0150530A3002730AA0010305A
:1000900055200330AA00E8305520AA0164305520CD
:1000A000AA010A3055202B085C28A9002C08A800BA
:1000B0002B08A700FB202708A700A3030319A01102
:1000C000240803196628230203186D282708031D36
:1000D000A011A0196D28303EBB280800AE00051005
:1000E00085108316051085100F30860583122E08A3
:1000F000A01898283E30A8008030E7203330AD00AB
:10010000AC201330A8008830E720AC206430E62013
:10011000AC206430E6202230AD00AC20283097209F
:100120000C30972006309720A0142E089828201411
:10013000AD00201CA6288510033C031CAB28AB2077
:100140000730A800D030E720031408002014FE3C3C
:100150000319B9288514201C201005140F308605BA
:100160002D08F03986040510AD0E2018AC28323069
:10017000E6202E081729A11B6E28080083169B0075
:1001800083161C141A089B0A172983169A001C153B
:1001900055309D00AA309D009C149C18CD281C1140
:1001A0009B0A172983178001840AFF3E031DD32869
:1001B0001729AA01A900FF30A907031CAA07031CDD
:1001C00017290330A800E530E720DB28A801F63E18
:1001D000A700A809031CF228FE300000A707031897
:1001E000ED28A7070000A80FEC2800002718F82822
:1001F0002718FA280800AC01AB011030AD00280D1B
:10020000AB0DAC0D2908AB022A08031C2A0FAC0267
:10021000031811292908AB072A0803182A0FAC076D
:100220000310A70DA80DAD0BFF282708172983136E
:10023000831203130800A00107309F008501860187
:10024000E33083168500FB30860081132030840064
:1002500060308312D320A03084005030D32020306F
:1002600084003030D2200515851505160130AA000E
:10027000F430DA20182054306E2072306E20613055
:100280006E206E306E2073306E2063306E207630BC
:100290006E2065306E2072306E2020306E2055301A
:1002A0006E204B306E2020306E2056306E202D3068
:1002B0006E2034306E208030A100C0302220773094
:1002C0006E206E206E202E306E2070306E206930D1
:1002D0006E2063306E2062306E2061306E2073308D
:1002E0006E2069306E2063306E202E306E206E30AE
:1002F0006E206C306E200730AA00D030DA20182033
:1003000041306E2044306E204A306E2055306E20D1
:1003100053306E2054306E203D306E2053306E20AE
:1003200065306E206C306E2065306E2063306E203C
:1003300074306E208030A100C030222053306E20F7
:1003400045306E204E306E2044306E203D306E20A1
:1003500043306E206F306E206E306E2074306E2011
:1003600069306E206E306E2075306E2065306E20E4
:100370000030BE20A6002608013A01390319C51233
:10038000031DC516861C092A0A30D9200301C51A87
:100390000130013A0319C512031DC5168D30222004
:1003A000A101C51EDA2952306E2043306E2035304F
:1003B0006E20E02952306E2043306E2036306E20A1
:1003C0000618E429BC22E029030106180130B20016
:1003D000030186180130B2050319F029BC22E42973
:1003E0008030A100C530222043306E206F306E2057
:1003F0006E306E2066306E2069306E2072306E2056
:100400006D306E2020306E206E206E206E206E20AB
:10041000C22986180C2A092A0030BE20A600260808
:10042000C51A013C03191B2A83169B010301831281
:10043000C51A0130C520C51E282A7F30BC001F30D8
:10044000BD000130BE20B9000230BE20C200322AF9
:10045000FF30BC00FF30BD000330BE20B9000430C7
:10046000BE20C2003908B6004208BF00C5151820DA
:100470007722E02AB401B30183108619831483180C
:100480004615831C461103018619013E4619013C9D
:1004900003190130031D0301B2003408A80033081A
:1004A000A7000130AA0013300620B20503195C2A08
:1004B000B30A0319B40A432A3408013A1330031962
:1004C0003306031D642A0B2DC51C722A8310461D9A
:1004D000831483184615831C46110230A80071301E
:1004E000E720762A0430A8004C30E720080080304E
:1004F000A100222053306E2079306E2073306E20A0
:100500003A306E203F083C2020306E206E20803034
:10051000A100C030222043306E206F306E206D303D
:100520006E203A306E2036083C2020306E206E203F
:10053000C51EAB2A8030A1008A3022200530A400DD
:100540003F082A208030A100C83022200730A400B4
:1005500036082A20BB2A8030A100883022200830AB
:10056000A4003F082A208030A100C8302220083093
:10057000A40036082A2008000A30D920B50A3330F2
:100580003502031CCC2AB501030105190130013ADB
:1005900003190511031D0515080001300618030194
:1005A000B2004308A70000300120B2050319DF2A7A
:1005B000C3030230D9208618DE2ADF2ACD2A08009C
:1005C0004515C51C45110515851503018618013013
:1005D000B200030106180130B2050319F22AC8302F
:1005E000BE004513030186180130B200030106184E
:1005F0000130B205030186190130B2050319012B40
:10060000F22A8619052BD32B122B0A30D92003018D
:1006100086180130B200030106180130B205031933
:10062000122BE02A0618782B8618172B162DC610C9
:100630004516C8303E02031D3B2BB430C4000130C8
:1006400006180301B2004408A70000300120B205DB
:1006500003192E2B0530D920C4031F2B013044026F
:1006600003183B2B0301C5190130013A0319C511C9
:10067000031DC5154517C51D4F2B851A472B3D0872
:1006800042020318452BC20A462BC2014E2B3C08DE
:10069000390203184D2BB90A4E2BB901602B851A6C
:1006A000592BC2080319562BC203582B3D08C20010
:1006B000602BB90803195E2BB903602B3C08B90005
:1006C0003908B6004208BF007722451F772B3E0845
:1006D000C300CD22C8303E02031D712BFA30C30087
:1006E000CD220D303E02031C772B0C30BE02D22BE4
:1006F0008618D22B451EB42B4512C51E9A2B0130ED
:10070000BE20A6002608390203198C2B013083165F
:100710009B0083123908C5200230BE20A60026089F
:1007200042020319992B023083169B008312420860
:10073000C520B42B0330BE20A600260839020319B9
:10074000A72B033083169B0083123908C520043081
:10075000BE20A600260842020319B42B04308316DB
:100760009B0083124208C520030146180130013A5C
:1007700003194610031D461483104618831483186A
:100780000516831C05128618D22B0511C51ACA2B13
:100790008825CB2B312505150618CF2B162D523069
:1007A000D920C32BE02AB401B3010130861903011B
:1007B000B2003408A8003308A700FF30AA00DC30DC
:1007C0000620B2050319E82BB30A0319B40AD52B86
:1007D0004510C510B408031DF32B1E303302031857
:1007E000F32BE02A2B2CB408031DFA2B2D303302F7
:1007F000031C062CB408031D062C3D3033020318DD
:10080000062C0830A8004D30E7202B2CB408031D1F
:100810000D2C5A303302031C1A2CB408031D1A2C59
:100820006F30330203181A2C45140530A80000302D
:10083000E7202B2CB408031D212C82303302031C2B
:100840002A2CB408031D2A2CB530330203182A2C95
:10085000C5142B2CE02A3708B8004008C100B701A6
:10086000C0010511C51C672C861D372C342C861938
:100870003A2C372C861D3D2C3A2C8619402C3D2CC9
:10088000861D432C402C0730A800D030E720831071
:100890008619831483180516831C05120301051A93
:1008A000013E8619013C031D562C4E2C0430A80035
:1008B0004C30E7203A22C017461DC0133A22401799
:1008C000461D40133A22C016461DC0126F2C3A2214
:1008D00083104619831483180516831C05123A22C7
:1008E0004016461D40123A22C015461DC0113A223C
:1008F0004015461D40113A22C014461DC0103A2230
:100900004014461D4010C51C8D2C3A22B717461DB9
:10091000B7133A223717461D37133A22B716461D2A
:10092000B7123A223716461D37123A22B715461D1E
:10093000B7113A223715461D37113A22B714461D12
:10094000B7103A223714461D3710451CA82C37170C
:1009500040084102031D0130B20037083802031D70
:100960000130B2040301C518013E4519013C031DC5
:100970000130B2040130C6180301B20403190A2D74
:100980001820451CCC2C52306E2043306E20353060
:100990006E2058306E20DB2CC51CD52C52306E20BA
:1009A00043306E2036306E20DB2C52306E204330C8
:1009B0006E2035306E2020306E2050306E20723028
:1009C0006E206F306E2074306E206F306E2063307A
:1009D0006E206F306E206C306E200330AA00E8303D
:1009E000DA20C51CF52CC512F62CC5163708B60042
:1009F0004008BF0018207722C6144008C2003708FC
:100A0000B9004614C51F4610C515C51C092DC512D1
:100A10000A2DC516E02A051585110330AA00E83015
:100A2000DA203808B7004108C000E02A1820523008
:100A30006E2065306E2073306E2074306E20613011
:100A40006E2072306E2074306E2001300618030163
:100A5000B200013086180301B2040319302D252D90
:100A60001E296A25391F6A25391B672546186A25FC
:100A7000461C6725421A6A25421E6725C2196A2547
:100A8000C21D672542196A25421D6725C2186A25BD
:100A9000C21C672542186A25421C6725B91A6A25B7
:100AA000B91E6725391A6A25391E6725B9196A25BD
:100AB000B91D672539196A25391D6725B9186A25B1
:100AC000B91C672539186A25391C6725080078255F
:100AD0006D2508006D2578250800FF30BB0000005B
:100AE00000000000000000000000BB0B6F2D08009C
:100AF0002030BA0000000F30BB00BB0B7D2D061567
:100B00000530BB00BB0B822D0611BA0B7A2D0800F5
:100B1000EC25EC25EC25EC25EC25EC25E525E5255B
:100B2000E225DF25DF25DF25461CEC25461CEC25CC
:100B3000E525E5254618EC254618EC25C21BE225DF
:100B4000C21FDF25421BE225421FDF25C21AE22514
:100B5000C21EDF25421AE225421EDF25C219E22508
:100B6000C21DDF254219E225421DDF25C218E225FC
:100B7000C21CDF254218E225421CDF25B91BE225F5
:100B8000B91FDF25391BE225391FDF25B91AE225F8
:100B9000B91EDF25391AE225391EDF25B919E225EC
:100BA000B91DDF253919E225391DDF25B918E225E0
:100BB000B91CDF253918E225391CDF250800E52599
:100BC000EC250800EC25E5250800E130BB0000001D
:100BD0000000BB0BE72D08001030BA0000000F30FA
:100BE000BB00BB0BF12D06150530BB00BB0BF62D72
:0A0BF0000611BA0BEE2D0800FC2DD3
:02400E00023F6F
:0A42000000000000000000000000B4
:00000001FF
